:020000040000fa
:080000003a02040000000000b8
:020000040000fa
:020000040002f8
:04afe000dfff00008f
:020000040000fa
:020000040002f8
:04afe400ffff00006b
:020000040000fa
:020000040002f8
:04afe80078ff0000ee
:020000040000fa
:020000040002f8
:04afec007dff0000e5
:020000040000fa
:020000040002f8
:04aff00078ff0000e6
:020000040000fa
:1000080000000000000000000000000000000000e8
:1000180032020000000000000000000000000000a4
:10002800000000000000000000000000f6030000cf
:1000380000000000000000000000000000000000b8
:10004800260400000000000000000000b2040000c8
:100058002e0500005e050000000000000000000002
:100068000000000000000000000000000000000088
:100078000000000000000000000000000000000078
:100088000000000000000000000000005204000012
:1000980082040000000000000000000000000000d2
:1000a8000000000000000000000000000000000048
:1000b8000000000000000000000000000000000038
:1000c8000000000000000000000000000000000028
:1000d8000000000000000000000000000000000018
:1000e8000000000000000000000000000000000008
:1000f80000000000000000000000000000000000f8
:1001080000000000000000000000000000000000e7
:1001180000000000000000000000000000000000d7
:1001280000000000ea0400000000000000000000d9
:1001380000000000000000000000000000000000b7
:1001480000000000000000000000000000000000a7
:100158000000000000000000000000000000000097
:100168000000000000000000000000000000000087
:100178000000000000000000000000000000000077
:100188000000000000000000000000000000000067
:10019800000000000000000098050000c4050000f1
:1001a800f005000000000000000000000000000052
:1001b8000000000000000000000000000000000037
:1001c8000000000000000000000000000000000027
:1001d8000000000000000000000000000000000017
:1001e8000000000000000000000000000000000007
:1001f80000000000000000000000000000000000f7
:1002080000000000000000000000000000000000e6
:1002180000000000000000000000000000000000d6
:1002280000000000000000000000000000000000c6
:1002380000000000000000000000000000000000b6
:1002480000000000000000000000000000000000a6
:100258000000000000000000000000000000000096
:100268000000000000000000000000000000000086
:0c0278000000000000000000000000007a
:020000040000fa
:10040000803e2000030007008100e900fcff3a0065
:1004100000000600831f7800c20320000400bc0017
:1004200066015100e0815900f23fb1000380b10044
:1004300006003500ee03090000000000423fb10055
:100440000380b100fbff3d001200b000223fb0006e
:10045000020035000280090000000000cf01780092
:10046000000006000020ef000220ef00c088a90075
:10047000004006000f002100b02e2100000188007e
:10048000000000000000eb00000778000c000900ed
:10049000002f78000007eb005420ef000e2eef0035
:1004a0001e2eef000000eb00a1212100e51d090038
:1004b0008018780040a7a900a1002000d0ff070005
:1004c000e0022000303a880044e7a90044c7a900b0
:1004d0004407a9004427a9004447a9004467a9008c
:1004e0004487a900300020000600fc003174200081
:1004f00082072000a3092000824878008348780002
:1005000080487800113a8000618070000600fc008d
:1005100021742000620420007305200082487800c6
:1005200083487800804878004427ef00e0022000ec
:10053000303a8800300020000d00fc0031742000ab
:1005400082072000a30920008248780083487800b1
:100550008048780000002000217420006204200000
:10056000730520008248780083487800804878002e
:1005700042a7ae00feff3700813e2000a0ff07002b
:1005800010c0b30086e6b70090c2b300c4e6b7005f
:1005900010eea90010cea900108ea90010aea9007f
:1005a000008ea900f0022000007088000070250075
:1005b0008070880010eea90010cea900108ea9004e
:1005c00010aea900008ea9000068a9004188a9000a
:1005d00041a8a90041c8a8002068a8000021ef0098
:1005e00002a1ef0004a1a8000481a80005e1a80071
:1005f0001061a8001021a90011e1a80011a1a90013
:1006000010a1a8001081a8000621ef000a21ef0028
:100610000ca1ef000ea1ef004408a9004428a90096
:100620004428a8000108a9002108a8002002a90068
:100630002022a9002042a90020a2a9002062a9002e
:100640002082a90020e2a9002102a9002122a900fc
:10065000700720004011880022a2a90022c2a90030
:1006600022e2a90021e2a8002182a9004588a90070
:1006700045a8a80045c8a8002168a8002828a80007
:1006800023e2a90023e2a9002342a8002362a900d3
:100690000188a9002188a8004608a9004628a800ca
:1006a0004648a8000e2eef00000ea800002ea8005d
:1006b000100ea800102ea8002c72ef002c12a8001b
:1006c000020eae002c12a9002c32a800022eae00a1
:1006d0002c32a9002c52a800120eae002c52a900f8
:1006e0002c72a800122eae002c72a9002cd2bf00d2
:1006f0000048b0002df2b7002cd2bf000049b00076
:100700002ef2b7002cd2bf00004ab0002ff2b70083
:100710002cd2bf00004bb00030f2b7002cd2bf008b
:10072000004cb00031f2b7002cd2bf00004db00039
:1007300032f2b7002cd2bf00004eb00033f2b70047
:100740000000eb00e1662100ff00090080587800fe
:100750003572ef003672ef002432ef002632ef00e0
:100760000000eb00e17621000801090080587800c4
:100770003772ef003872ef004872ef0070c0b300bc
:100780004852e3000a003e0048d2bf000080fb0050
:10079000c200dd00e064210000814000f0ff2f0076
:1007a000f1ff2f000089be004872ec00f3ff390012
:1007b0000000eb00e1442100ff00090080187800f0
:1007c0004b72ef004c72ef006103070071050700e8
:1007d0007105070014eea90014cea900148ea9001b
:1007e00014aea900048ea90020013700ff3ffc00d1
:1007f0004200f8003600f8004400f8008e1f780030
:100800000e0020000d000900be1f78003200f80025
:100810000100fc000068a90012aeaa0010aea900f9
:10082000ff3ffc003200f900ae0120000d0009007e
:100830004f1778004f0778004400f9003600f900a0
:100840004200f9000100fc0000400600ff3ffc00f0
:100850004200f8003600f8004400f8008e1f7800cf
:100860000e0020000d000900be1f78003200f800c5
:100870000100fc000108a900ff3ffc003200f90064
:10088000ae0120000d0009004f1778004f077800d7
:100890004400f9003600f9004200f9000100fc00b4
:1008a00000400600ff3ffc004200f8003600f80060
:1008b0004400f8008e1f78000e0020000d00090093
:1008c000be1f78003200f8000100fc000368a90098
:1008d0001421ef002368a800ff3ffc003200f9005c
:1008e000ae0120000d0009004f1778004f07780077
:1008f0004400f9003600f9004200f9000100fc0054
:1009000000400600ff3ffc004200f8003600f800ff
:100910004400f8008e1f78000e0020000d00090032
:10092000be1f78003200f8000100fc000388a90017
:100930001821ef002388a800ff3ffc003200f900d7
:10094000ae0120000d0009004f1778004f07780016
:100950004400f9003600f9004200f9000100fc00f3
:1009600000400600ff3ffc004200f8003600f8009f
:100970004400f8008e1f78000e0020000d000900d2
:10098000be1f78003200f8000100fc000168a900d9
:100990003572ec0035d2bf008080fb003011800042
:1009a000e266210080707900ff3ffc003200f90010
:1009b000ae0120000d0009004f1778004f077800a6
:1009c0004400f9003600f9004200f9000100fc0083
:1009d00000400600ff3ffc004200f8003600f8002f
:1009e0004400f8008e1f78000e0020000d00090062
:1009f000be1f78003200f8000100fc000828a900a2
:100a00002242ae000300370014cea8002242a90003
:100a10000100370014cea9002222ae0003003700e7
:100a200014eea8002222a9000100370014eea9004c
:100a3000ff3ffc003200f900ae0120000d0009006c
:100a40004f1778004f0778004400f9003600f9008e
:100a50004200f9000100fc0000400600ff3ffc00de
:100a60004200f8003600f8004400f8008e1f7800bd
:100a70000e0020000d000900be1f78003200f800b3
:100a80000100fc000188a900128eaa00108ea900a6
:100a9000ff3ffc003200f900ae0120000d0009000c
:100aa0004f1778004f0778004400f9003600f9002e
:100ab0004200f9000100fc0000400600ff3ffc007e
:100ac0004200f8003600f8004400f8008e1f78005d
:100ad0000e0020000d000900be1f78003200f80053
:100ae0000100fc0001a8a9004b72ec004bd2bf0032
:100af0000080fb0000004000e1442100021880005b
:100b000002b07800ff3ffc003200f900ae01200087
:100b10000d0009004f1778004f0778004400f900d6
:100b20003600f9004200f9000100fc000040060018
:100b3000ff3ffc004200f8003600f8004400f800d7
:100b40008e1f78000e0020000d000900be1f7800e7
:100b50003200f8000100fc000bc8a900ff3ffc00b8
:100b60003200f900ae0120000d0009004f17780097
:100b70004f0778004400f9003600f9004200f90000
:100b80000100fc0000400600ff3ffc004200f800ae
:100b90003600f8004400f8008e1f78000e00200098
:100ba0000d000900be1f78003200f8000100fc00b3
:100bb0000be8a900ff3ffc003200f900ae01200065
:100bc0000d0009004f1778004f0778004400f90026
:100bd0003600f9004200f9000100fc000040060068
:100be000ff3ffc004200f8003600f8004400f80027
:100bf0008e1f78000e0020000d000900be1f780037
:100c00003200f8000100fc000c08a900ff3ffc00c6
:100c10003200f900ae0120000d0009004f177800e6
:100c20004f0778004400f9003600f9004200f9004f
:100c30000100fc000040060036d2bf003552e30040
:100c4000070032003672ec0036d2bf000080fb0095
:100c5000e166210060c0780039f2b700010037007a
:100c600039f2ef00000006000000060030088000a6
:100c7000209188005008800030918800eeff070026
:100c800033d2bf003952e30006003600e0cfb30094
:100c90003952b50001003900010037003a72ef0007
:100ca000be01370039f2ae00370037003a72ef006c
:100cb00039d2bf002d52b50005003a0039d2bf002d
:100cc0003af2b7003bf2ef003cf2ef002d003700a4
:100cd00039d2bf002e52b50005003a0039d2bf000c
:100ce0003af2b7003df2ef003ef2ef002500370088
:100cf00039d2bf002f52b50005003a0039d2bf00eb
:100d00003af2b7003ff2ef0040f2ef001d0037006b
:100d100039d2bf003052b50005003a0039d2bf00c9
:100d20003af2b70041f2ef0042f2ef00150037004f
:100d300039d2bf003152b50004003a0039d2bf00a9
:100d40003af2b70043f2ef000e00370039d2bf008d
:100d50003252b50004003a0039d2bf003af2b7006f
:100d600044f2ef000700370039d2bf003352b5001c
:100d700004003a0039d2bf003af2b70045f2ef0062
:100d800046f2ef00850137003a52e20002003a00d5
:100d900082013700810137003ad2bf002d52b500e1
:100da0004a003a0000e0ef003b52e30003003a0043
:100db00039d2bf003bf2b7004300370039d2bf0041
:100dc0003cf2b7003bd2bf0051c1b30080cf10004e
:100dd0002300360047d2bf008080fb0020062000a1
:100de00001005000800078003bd2bf000080fb0073
:100df000810f50001a003e003772ec0037d2bf005e
:100e00000081fb00e17621002dd2bf0000f17800c7
:100e10003772ec0047d2bf000080fb008007b000b3
:100e2000e09088003bd2bf000080fb001c12b500a0
:100e300071232100914078008180fb00e27621003f
:100e4000807079003772ec0037d2bf000081fb0060
:100e5000e17621003cd2bf0000f178001900370094
:100e60003bd2bf0051c1b30080cf10000300360059
:100e7000f0c6b3003b52b500120039003772ec00e7
:100e800037d2bf000081fb00e17621002dd2bf00e8
:100e900000f178003772ec0037d2bf000081fb0010
:100ea000e17621003bd2bf0000f178003772ec0000
:100eb00037d2bf000081fb00e17621003cd2bf00a9
:100ec00000f178003bf2ef00340137003ad2bf0066
:100ed0002e52b5004a003a0000e0ef003d52e30018
:100ee00003003a0039d2bf003df2b700430037009b
:100ef00039d2bf003ef2b7003dd2bf0051c1b300ae
:100f000080cf10002300360047d2bf008080fb0056
:100f10002006200001005000800078003dd2bf0074
:100f20000080fb00810f50001a003e003772ec0079
:100f300037d2bf000081fb00e17621002ed2bf0036
:100f400000f178003772ec0047d2bf000080fb0050
:100f50008007b000e09088003dd2bf000080fb0019
:100f60001c12b50071232100914078008180fb00a4
:100f7000e2762100807079003772ec0037d2bf0032
:100f80000081fb00e17621003ed2bf0000f1780035
:100f9000190037003dd2bf0051c1b30080cf10000f
:100fa00003003600f0c6b3003d52b5001200390010
:100fb0003772ec0037d2bf000081fb00e1762100e0
:100fc0002ed2bf0000f178003772ec0037d2bf009c
:100fd0000081fb00e17621003dd2bf0000f17800e6
:100fe0003772ec0037d2bf000081fb00e1762100b0
:100ff0003ed2bf0000f178003df2ef00e70037007d
:101000003ad2bf002f52b50049003a0000e0ef008d
:101010003f52e30003003a0039d2bf003ff2b7006d
:101020004200370039d2bf0040f2b7003fd2bf00c4
:1010300051c1b30080cf10002300360047d2bf005b
:101040008080fb0020062000010050008000780016
:101050003fd2bf000080fb00810f50001a003e000d
:101060003772ec0037d2bf000081fb00e17621002f
:101070002fd2bf0000f178003772ec0047d2bf00da
:101080000080fb008007b000e09088003fd2bf00e6
:101090000080fb001c12b5007123210091407800f4
:1010a0008180fb00e2762100807079003772ec00cd
:1010b00037d2bf000081fb00e176210040d2bf00a3
:1010c00000f17800190037003fd2bf0051c1b300d2
:1010d00080cf100003003600f0c6b3003f52b500c9
:1010e000120039003772ec0037d2bf000081fb00dc
:1010f000e17621002fd2bf0000f178003772ec00ba
:1011000037d2bf000081fb00e17621003fd2bf0053
:1011100000f178003772ec0037d2bf000081fb008d
:10112000e176210040d2bf0000f178009b0037003b
:101130003ad2bf003052b50051003a0000e0ef0053
:101140004152e30003003a0039d2bf0041f2b70038
:101150004a00370039d2bf0042f2b70020c3b300c3
:101160004152e3001a003a003772ec0037d2bf0058
:101170000081fb00e176210030d2bf0000f1780051
:101180003772ec0037d2bf000080fb00b2072000ae
:10119000e176210002f078003772ec0037d2bf0010
:1011a0000080fb0002002000e176210002f07800c0
:1011b00042d2bf0047f2b700d0c0b3004752b500db
:1011c00002003900c0c0b30047f2b7002b0037005f
:1011d00020c4b3004152e30016003a004252e2003c
:1011e00001003a004772ef003772ec0037d2bf00bf
:1011f0000081fb00e176210030d2bf0000f17800d1
:101200003772ec0037d2bf000081fb00e17621008d
:1012100041d2bf0000f178003772ec0037d2bf0036
:101220000081fb00e176210042d2bf0000f178008e
:10123000120037003772ec0037d2bf000081fb008c
:10124000e176210030d2bf0000f178003772ec0067
:1012500037d2bf000081fb00e176210041d2bf0000
:1012600000f178003772ec0037d2bf000081fb003c
:10127000e176210042d2bf0000f17800470037003c
:101280003ad2bf003152b50012003a0000e0ef0040
:101290004352e3000e003a0039d2bf0043f2b700d8
:1012a0003772ec0037d2bf000081fb00e1762100ed
:1012b00031d2bf0000f178003772ec0037d2bf00a6
:1012c0000081fb00e176210043d2bf0000f17800ed
:1012d000320037003ad2bf003252b50012003a0055
:1012e00000e0ef004452e3000e003a0039d2bf00a4
:1012f00044f2b7003772ec0037d2bf000081fb0028
:10130000e176210032d2bf0000f178003772ec00a4
:1013100037d2bf000081fb00e176210044d2bf003c
:1013200000f178001d0037003ad2bf003352b500fb
:101330001a003a0000e0ef004552e30003003a00d3
:1013400039d2bf0045f2b7001400370039d2bf00d0
:1013500046f2b7003772ec0037d2bf000081fb00c5
:10136000e176210033d2bf0000f178003772ec0043
:1013700037d2bf000081fb00e176210045d2bf00db
:1013800000f178003772ec0037d2bf000081fb001b
:10139000e176210046d2bf0000f178004a32af006a
:1013a0003900070080c0b3004952b5002300310066
:1013b0002291800033918000409180005191800003
:1013c000800f5100818f5900100039002bf2a800c6
:1013d0004952e20001003a000b00370010c0b30090
:1013e0004952e30001003a000700370020c0b30073
:1013f0004952e30001003a000300370030c0b30057
:101400004952e30000003a001f00070027f2ae0037
:10141000090037002432ef002632ef000621ef00ea
:101420000a21ef002032ef000080eb00e164210090
:101430000f000900801878000600370027f2ae0080
:10144000040037002432ef002632ef000621ef00bf
:101450000a21ef0037d2bf003852e3000900320002
:101460000188af00070037003872ec0038d2bf00a7
:101470000080fb00e176210060c078000080fb0066
:1014800020118800f9fd370049f2ef002bf2a80087
:101490004872ef0070c0b3004852e30018003e00ed
:1014a00048d2bf000080fb00c200dd00e0642100e4
:1014b000008040001000be000001be00409180008e
:1014c00051918000800f5100818f59000a00310036
:1014d00048d2bf000080fb00c200dd00e0642100b4
:1014e000008040001000be004091880051918800ab
:1014f00048d2bf0049f2b7004872ec00e5ff39005e
:101500004a32a900000006002232ef002032ef002c
:101510004a32a8004872ef0070c0b3004852e3009e
:101520000a003e0048d2bf000080fb00c200dd0080
:10153000e064210000814000f0ff2f00f1ff2f0048
:101540000089be004872ec00f3ff3900000006007d
:101550004eb2ef00a0c72500809288005098250069
:101560009092880040812500a0928800906a250012
:10157000b092880030542500c0928800303e25008b
:10158000d092880090282500e09288005013250012
:10159000f092880060fe240000938800c0e92400d7
:1015a0001093880080d524002093880090c12400e7
:1015b00030938800f0ad240040938800a09a240066
:1015c00050938800a087240060938800f074240062
:1015d00070938800906224008093880080502400db
:1015e00090938800b03e2400a0938800302d240002
:1015f000b0938800f01b2400c0938800000b2400e7
:10160000d093880050fa2300e0938800e0e923009b
:10161000f0938800c0d9230000948800e0c923001b
:101620001094880040ba230020948800e0aa230088
:1016300030948800c09b230040948800e08c2300f5
:1016400050948800307e230060948800d06f23007f
:1016500070948800a061230080948800b053230018
:1016600090948800f0452300a094880070382300ef
:10167000b0948800202b2300c0948800101e230003
:10168000d094880040112300e09488009004230047
:10169000f094880020f8220000958800e0eb2200fa
:1016a00010958800d0df220020958800f0d322001a
:1016b0003095880050c8220040958800d0bc220098
:1016c0005095880080b122006095880070a62200a5
:1016d00070958800809b220080958800c090220031
:1016e0009095880020862200a0958800c07b22006b
:1016f000b095880080712200c09588006067220044
:10170000d0958800805d2200e0958800c0532200bb
:10171000f0958800204a220000968800b040220000
:10172000109688006037220020968800402e220004
:10173000309688004025220040968800601c2200d8
:1017400050968800b013220060968800200b22007b
:1017500070968800b00222008096880060fa21000e
:101760009096880040f22100a096880030ea21007f
:10177000b096880050e22100c096880090da2100df
:10178000d0968800e0d22100e096880060cb21004e
:10179000f0968800f0c3210000978800b0bc2100bb
:1017a0001097880080b521002097880080ae210026
:1017b0003097880090a7210040978800b0a02100b2
:1017c00050978800009a210060978800609321005c
:1017d00070978800e08c2100809788008086210027
:1017e0009097880030802100a0978800007a21001f
:1017f000b0978800f0732100c0978800f06d210039
:10180000d097880000682100e0978800406221009e
:10181000f0978800805c210000988800e056210045
:10182000109888006051210020988800f04b21001a
:10183000309888009046210040988800504121004f
:1018400050988800203c21006098880010372100c3
:10185000709888001032210080988800202d210087
:101860009098880040282100a098880080232100bb
:10187000b0988800d01e2100c0988800301a21003e
:10188000d0988800a0152100e09888002011210040
:10189000f0988800c00c2100009988007008210091
:1018a000109988002004210020998800f0ff200072
:1018b00030998800d0fb200040998800c0f72000b4
:1018c00050998800d0f3200060998800e0ef200054
:1018d0007099880000ec20008099880030e8200092
:1018e0009099880070e42000a0998800c0e0200052
:1018f000b099880020dd2000c099880090d9200090
:10190000d099880010d62000e0998800a0d220004d
:10191000f099880040cf2000009a8800e0cb20009a
:10192000109a8800a0c82000209a880060c5200076
:10193000309a880030c22000409a880010bf2000f2
:10194000509a880000bc2000609a88004eb3ef00d7
:10195000302c2a00809a880060a42900909a880080
:1019600020632900a09a8800a0232900b09a88004b
:10197000d0e52800c09a8800a0a92800d09a880045
:10198000006f2800e09a8800f0352800f09a88005f
:1019900070fe2700009b880050c82700109b88001d
:1019a000b0932700209b880070602700309b880040
:1019b000802e2700409b8800f0fd2600509b880069
:1019c000a0ce2600609b8800a0a02600709b880007
:1019d000c0732600809b880020482600909b8800ca
:1019e000a01d2600a09b880040f42500b09b880025
:1019f000f0cb2500c09b8800c0a42500d09b8800a8
:101a0000907e2500e09b880060592500f09b8800af
:101a100030352500009c880000122500109c8800ad
:101a2000b0ef2400209c880050ce2400309c880019
:101a3000c0ad2400409c8800208e2400509c88006b
:101a4000506f2400609c880050512400709c8800d6
:101a500020342400809c8800b0172400909c8800cb
:101a600000fc2300a09c880000e12300b09c8800bb
:101a7000d0c62300c09c880040ad2300d09c8800c5
:101a800060942300e09c8800207c2300f09c880068
:101a900090642300009d8800a04d2300109d8800c5
:101aa00040372300209d880080212300309d88003e
:101ab000500c2300409d8800b0f72200509d880004
:101ac000a0e32200609d880020d02200709d880045
:101ad00010bd2200809d880090aa2200909d880061
:101ae00080982200a09d8800f0862200b09d88008a
:101af000e0752200c09d880030652200d09d8800de
:101b000000552200e09d880040452200f09d88009d
:101b1000e0352200009e8800f0262200109e8800fa
:101b200060182200209e8800300a2200309e880023
:101b300060fc2100409e8800f0ee2100509e88004d
:101b4000e0e12100609e880020d52100709e880081
:101b5000c0c82100809e8800b0bc2100909e8800f3
:101b6000f0b02100a09e880080a52100b09e8800d2
:101b7000509a2100c09e8800808f2100d09e88004e
:101b8000f0842100e09e8800b07a2100f09e880059
:101b9000a0702100009f8800f0662100109f88003f
:101ba000705d2100209f880030542100309f880004
:101bb000304b2100409f880070422100509f8800d8
:101bc000f0392100609f8800a0312100709f8800bb
:101bd00090292100809f8800b0212100909f8800db
:101be000101a2100a09f880090122100b09f880049
:101bf000500b2100c09f880040042100d09f880026
:101c000060fd2000e09f8800b0f62000f09f880073
:101c100030f0200000a08800d0e9200010a088004b
:101c2000a0e3200020a08800a0dd200030a08800d4
:101c3000c0d7200040a0880010d2200050a088000b
:101c400080cc200060a0880020c7200070a0880001
:101c5000e0c1200080a08800c0bc200090a08800c7
:101c6000c0b72000a0a08800e0b22000b0a088008b
:101c700030ae2000c0a0880090a92000d0a088002d
:101c800010a52000e0a08800b0a02000f0a08800ef
:101c9000809c200000a188005098200010a188009e
:101ca0005094200020a188006090200030a188007e
:101cb000908c200040a18800e088200050a188007e
:101cc0004085200060a18800c081200070a18800ac
:101cd000507e200080a18800f07a200090a188002a
:101ce000b0772000a0a1880090742000b0a18800e7
:101cf00070712000c0a18800706e2000d0a1880003
:101d0000906b2000e0a18800b0682000f0a188005e
:101d1000f065200000a288004063200010a2880027
:101d2000a060200020a28800105e200030a2880061
:101d3000905b200040a288003059200050a288000b
:101d4000d056200060a288004872ef00f0c7b300b0
:101d50004852e3000e003e0048d2bf000080fb0066
:101d600000004000e1342100608078004300de0084
:101d700081242100914078008180fb008180400017
:101d8000e2342100803079004872ec00efff390026
:101d9000000006000000060000000600ffff3700fc
:020000040000fa
:101da0001a1200000600000080000000201200004f
:101db0000400000080000000241200000800000061
:101dc000800000002c1200002200000080000000b3
:101dd0004e12000000040000800000004e160000bb
:101de00020000000800000006e1600000a020000c3
:081df00080000000000000006b
:00000001FF
